:020000040000FA
:1000000000020400000000006A0300006A03000010
:100010006A0300006A0300006A0300006A0300002C
:100020006A0300006A0300006A0300006A0300001C
:100030006A0300006A0300006A0300006A0300000C
:100040006A0300006A0300006A0300006A030000FC
:100050006A0300006A0300006A030000BC0200009B
:100060006A0300006A0300006A0300006A030000DC
:100070006A0300006A0300006A0300006A030000CC
:100080006A0300006A0300006A0300006A030000BC
:100090006A0300006A0300006A0300006A030000AC
:1000A0006A0300006A0300006A0300006A0300009C
:1000B0006A0300006A0300006A0300006A0300008C
:1000C0006A0300006A0300006A0300006A0300007C
:1000D0006A0300006A0300006A0300006A0300006C
:1000E0006A0300006A0300006A0300006A0300005C
:1000F0006A0300006A0300006A0300006A0300004C
:100100006A0300006A0300006A0300006A0300003B
:100110006A0300006A0300006A0300006A0300002B
:100120006A0300006A0300006A0300006A0300001B
:100130006A0300006A0300006A0300006A0300000B
:100140006A0300006A0300006A0300006A030000FB
:100150006A0300006A0300006A0300006A030000EB
:1001600062030000E8020000FFFFFF00FFFFFF0046
:10017000FFFFFF00FFFFFF00FFFFFF00FFFFFF008B
:10018000FFFFFF00FFFFFF00FFFFFF00FFFFFF007B
:10019000FFFFFF00FFFFFF00FFFFFF00FFFFFF006B
:1001A000FFFFFF00FFFFFF00FFFFFF00FFFFFF005B
:1001B000FFFFFF00FFFFFF00FFFFFF00FFFFFF004B
:1001C000FFFFFF00FFFFFF00FFFFFF00FFFFFF003B
:1001D000FFFFFF00FFFFFF00FFFFFF00FFFFFF002B
:1001E000FFFFFF00FFFFFF00FFFFFF00FFFFFF001B
:1001F000FFFFFF00FFFFFF00FFFFFF00FFFFFF000B
:10020000FFFFFF00FFFFFF006A0300006A0300001A
:100210006A0300006A0300006A0300006A0300002A
:100220006A0300006A0300006A0300006A0300001A
:100230006A0300006A0300006A0300006A0300000A
:100240006A0300006A0300006A0300006A030000FA
:100250006A0300006A0300006A0300006A030000EA
:100260006A0300006A0300006A0300006A030000DA
:100270006A0300006A0300006A0300006A030000CA
:100280006A0300006A0300006A0300006A030000BA
:100290006A0300006A0300006A0300006A030000AA
:1002A0006A0300006A0300006A0300006A0300009A
:1002B0006A0300006A0300006A0300006A0300008A
:1002C0006A0300006A0300006A0300006A0300007A
:1002D0006A0300006A0300006A0300006A0300006A
:1002E0006A0300006A0300006A0300006A0300005A
:1002F0006A0300006A0300006A0300006A0300004A
:100300006A0300006A0300006A0300006A03000039
:100310006A0300006A0300006A0300006A03000029
:100320006A0300006A0300006A0300006A03000019
:100330006A0300006A0300006A0300006A03000009
:100340006A0300006A0300006A0300006A030000F9
:100350006A0300006A0300006A0300006A030000E9
:100360006A0300006A030000FFFFFF00FFFFFF00B9
:10037000FFFFFF00FFFFFF00FFFFFF00FFFFFF0089
:10038000FFFFFF00FFFFFF00FFFFFF00FFFFFF0079
:10039000FFFFFF00FFFFFF00FFFFFF00FFFFFF0069
:1003A000FFFFFF00FFFFFF00FFFFFF00FFFFFF0059
:1003B000FFFFFF00FFFFFF00FFFFFF00FFFFFF0049
:1003C000FFFFFF00FFFFFF00FFFFFF00FFFFFF0039
:1003D000FFFFFF00FFFFFF00FFFFFF00FFFFFF0029
:1003E000FFFFFF00FFFFFF00FFFFFF00FFFFFF0019
:1003F000FFFFFF00FFFFFF00FFFFFF00FFFFFF0009
:100400008F8021000E7F24000E0188000000000074
:10041000000020000000E000020032000001200087
:10042000200288000E000700A0C22000010020006A
:10043000810F70000100320014000700000020004E
:100440000000E00002003200000002000000000096
:10045000880B0200000000000040DA000000FE00EF
:100460004440A900008020000000E00003003200AA
:1004700000002000A00188004440A8000000060001
:100480008A1F78008B1F7800000006009101880009
:10049000800478000000EB001A003700E28444007A
:1004A00032A0B4009905BA00E284440032A0B4003E
:1004B0009906BA00E284440032A0B4000006EB00C2
:1004C000476FDE00FD07B200636CE10003003A00F5
:1004D000EBFF07000000EB000A003700606CE10052
:1004E00004003A00005DEB008B05E900FDFF3E00D3
:1004F000040037006168E100010032000086EB0073
:100500000B00070019C7BA001905BA000E04E00075
:1005100003003A000A00E000E0FF3A000000060095
:10052000FE07B2009E0188008A047800F5FF3700BC
:10053000395DBA008B05E9000C003200295DBA0074
:100540008B05E900080032000C00E00003003A00CF
:10055000E284440032A0B400F5FF370019DDBA0090
:100560008B05E900FAFF3A008904E800E1844400C1
:1005700032A0B40000000600801F78000000FA00DE
:1005800085A0A90004C8BF000004E00006003A00EE
:10059000001880000040880050502000401988005A
:1005A0002023A800040037000018800010408800B5
:1005B000404020004019880004C8BF000004A20089
:1005C00004E8B7000080FA004F0078000040060001
:1005D0003600F800809FBE00829FBE00849FBE0050
:1005E000869FBE000400FA008DE0A9000140800053
:1005F000010F780011408000110798002023A80007
:10060000304080008000400080802000008040005A
:100610001E087800304080000020B00080004000BC
:1006200080802000008040001E087800304080005C
:1006300000004000800078008080200000804000A2
:1006400082002100800078000020200023000700A5
:10065000000F7800304080000000400080007800EB
:1006600080802000008040008240210080007800CF
:10067000002020001900070010079800304080007B
:100680000000E9003040880031408000F01F200069
:1006900000806000304088001E007800C01F880085
:1006A0001E009000B01F88000080FA004F03BE00BB
:1006B0004F02BE004F01BE004F00BE003600F900E1
:1006C000004006000000FA008DC0A9000080FA007A
:1006D000004006000040DA000000FE004400F80080
:1006E000040F2000240288000000E9001201C3006A
:1006F000008008000200000031027800B202780099
:100700001201C0000000CD004400F9000000060006
:1007100000000000000000000000000000000000D9
:1007200000000000000000000000000000000000C9
:1007300000000000000000000000000000000000B9
:1007400000000000000000000000000000000000A9
:100750000000000000000000000000000000000099
:1007600000000000FFFF000000000000000000008B
:10077000FFFF0000FFFF000000000000000000007D
:10078000FFFF00000000000001000000000000006A
:100790000000000001000000010000000000000057
:1007A0000100000002000000010000000000000045
:1007B0000200000002000000000000000100000034
:1007C0000300000000000000FFFF00000100000027
:1007D00001000000FDFF0000FEFF0000010000001E
:1007E000FEFF0000FBFF0000FFFF0000FFFF000016
:1007F000FAFF0000FCFF000000000000FCFF00000A
:10080000FAFF0000FFFF000000000000FBFF0000F7
:10081000FDFF00000300000000000000FCFF0000DE
:100820000300000006000000FFFF000001000000C0
:100830000A000000050000000000000009000000A0
:100840000C00000002000000030000000D0000008A
:1008500006000000FDFF0000070000000A00000085
:10086000FCFF0000FCFF000007000000FFFF00008D
:10087000F3FF0000FDFF000002000000F1FF000098
:10088000F0FF0000FFFF0000F7FF0000E9FF00009D
:10089000F7FF000000000000EEFF0000EDFF000089
:1008A00003000000FDFF0000EDFF0000FFFF00005F
:1008B0000D000000FAFF0000F9FF00001500000025
:1008C00010000000FBFF00000F00000022000000ED
:1008D0000900000004000000230000001C000000CC
:1008E000FFFF0000120000002600000005000000CD
:1008F000F9FF00001A00000011000000E9FF0000ED
:10090000FBFF000012000000EBFF0000D9FF000019
:1009100000000000F8FF0000CAFF0000DFFF000039
:1009200000000000D8FF0000C4FF0000F7FF000037
:10093000F7FF0000C6FF0000E2FF00001200000009
:10094000EBFF0000D6FF0000160000001F000000B3
:10095000E8FF00000700000043000000180000004E
:10096000FBFF0000420000004D00000007000000F7
:1009700020000000610000002B000000FBFF0000D1
:10098000420000004B000000EFFF0000FDFF0000F0
:100990004400000001000000BDFF0000080000004E
:1009A00015000000A8FF0000B3FF00000A000000CF
:1009B000C5FF000077FF0000D3FF0000F3FF000039
:1009C00081FF000091FF000007000000CDFF000044
:1009D0007BFF0000F0FF00002C000000B4FF0000CF
:1009E000CAFF0000610000002D000000CCFF0000E5
:1009F00052000000A1000000140000001D000000D3
:100A0000C600000088000000000000008300000015
:100A1000D80000002100000008000000BB0000001A
:100A200067000000AAFF000027000000850000000A
:100A3000A3FF00006AFF000036000000DEFF000098
:100A4000F6FE000083FF00000900000012FF000016
:100A5000CFFE0000DAFF00009FFF00009FFE0000B5
:100A600059FF00002F00000031FF0000F0FE0000E1
:100A7000570000004700000023FF00000E000000A8
:100A80003D01000022000000C0FF00007D010000C9
:100A900081010000FBFF0000F1000000690200007E
:100AA000EB0000001D000000200200000F0200000B
:100AB000C2FF00009D000000680200003900000035
:100AC000AAFE0000210100000201000077FD0000E5
:100AD00047FE0000EF000000C0FD00000AFB000020
:100AE000DAFE000026FF00004EF9000085FA000043
:100AF00016000000DBFA000007F5000018FE0000F9
:100B00004D01000068F0000067F20000C71D000002
:100B1000663B0000C61D000068F2000069F000009E
:100B20004D01000019FE000009F50000DCFA00008C
:100B30001600000086FA000051F9000026FF0000B0
:100B4000DAFE00000CFB0000C1FD0000EF00000019
:100B500048FE000079FD00000201000021010000B4
:100B6000ABFE000039000000670200009C0000009E
:100B7000C2FF00000E0200001E0200001D00000067
:100B8000EA00000067020000F0000000FBFF000028
:100B90007F0100007C010000C1FF00002200000076
:100BA0003C0100000E00000025FF0000470000008F
:100BB00056000000F2FE000032FF00002E00000090
:100BC0005AFF0000A1FE00009FFF0000DBFF0000B5
:100BD000D1FE000013FF00000900000084FF0000A8
:100BE000F8FE0000DEFF0000360000006BFF000092
:100BF000A4FF00008400000027000000ABFF0000FD
:100C000067000000B900000008000000210000009B
:100C1000D6000000820000000000000086000000F6
:100C2000C40000001D00000014000000A00000002F
:100C300051000000CDFF00002D000000600000000A
:100C4000CBFF0000B5FF00002C000000F0FF00000B
:100C50007CFF0000CEFF00000700000092FF0000B4
:100C600082FF0000F4FF0000D4FF000079FF0000C5
:100C7000C6FF00000A000000B3FF0000A9FF00004B
:100C80001500000008000000BEFF00000100000089
:100C900043000000FDFF0000EFFF00004A000000DD
:100CA00041000000FBFF00002A000000600000007F
:100CB00020000000070000004C0000004100000080
:100CC000FBFF0000180000004200000007000000C9
:100CD000E8FF00001E00000016000000D7FF000023
:100CE000EBFF000011000000E2FF0000C7FF000062
:100CF000F7FF0000F7FF0000C5FF0000D8FF00006D
:100D000000000000E0FF0000CBFF0000F8FF000043
:100D100000000000DAFF0000ECFF000012000000FD
:100D2000FBFF0000EAFF0000100000001A000000B6
:100D3000FAFF00000500000025000000120000007E
:100D4000FFFF00001C000000220000000400000063
:100D500009000000210000000F000000FBFF000060
:100D60000F00000014000000F9FF0000FAFF00006F
:100D70000D000000FFFF0000EDFF0000FDFF000080
:100D800003000000EEFF0000EEFF00000000000086
:100D9000F7FF0000E9FF0000F8FF0000FFFF000080
:100DA000F0FF0000F1FF000002000000FDFF000066
:100DB000F3FF0000FFFF000007000000FCFF000041
:100DC000FCFF00000A00000006000000FEFF00001B
:100DD000060000000D0000000300000002000000FB
:100DE0000B000000080000000000000005000000EB
:100DF0000A00000001000000FFFF000006000000E4
:100E000003000000FCFF00000000000003000000E1
:100E1000FDFF0000FBFF000000000000FFFF0000DE
:100E2000FAFF0000FDFF000000000000FCFF0000D2
:100E3000FBFF0000FFFF0000FFFF0000FCFF0000C1
:100E4000FEFF000001000000FFFF0000FEFF0000A9
:100E50000100000001000000FFFF00000000000092
:100E6000030000000100000000000000020000007C
:100E7000020000000000000001000000020000006D
:100E8000010000000000000001000000010000005F
:100E90000000000000000000010000000000000051
:100EA000FFFF00000000000000000000FFFF000046
:100EB000000000000000000000000000FFFF000034
:100EC0000000000000000000000000000000000022
:100ED0000000000000000000000000000000000012
:100EE0000000000000000000000000000000000002
:100EF00000000000000000000000000000000000F2
:100F000000000000000000000000000000000000E1
:100F100000000000000000000000000000000000D1
:100F200000000000000000000000000000000000C1
:100F300000000000000000000000000000000000B1
:100F400000000000000000000000000000000000A1
:100F50000000000000000000000000000000000091
:100F60000000000000000000FFFF00000000000083
:100F700000000000FFFF0000FFFF00000000000075
:100F800000000000FFFF0000FFFF00000000000065
:100F9000FFFF0000FFFF0000000000000000000055
:100FA000FFFF000000000000010000000000000042
:100FB000FFFF00000200000002000000000000002F
:100FC000020000000300000001000000000000001B
:100FD0000400000003000000000000000200000008
:100FE0000400000001000000FFFF000003000000FB
:100FF00002000000FDFF0000FFFF000002000000F3
:10100000FDFF0000FAFF000000000000FFFF0000ED
:10101000F8FF0000FBFF000000000000FAFF0000E6
:10102000F7FF0000FFFF0000FFFF0000F7FF0000D8
:10103000FBFF000003000000FDFF0000F9FF0000BF
:101040000400000006000000FCFF0000010000009A
:101050000C00000005000000FFFF00000C00000075
:101060000E00000001000000060000001200000059
:1010700008000000FFFF00000C0000000E00000050
:10108000FCFF0000FEFF00000D000000000000005B
:10109000F2FF00000100000004000000EEFF00006D
:1010A000EFFF000001000000F4FF0000E3FF00007C
:1010B000F6FF0000FEFF0000E6FF0000E8FF000072
:1010C00002000000F6FF0000E4FF0000FDFF00004A
:1010D0000B000000F1FF0000F5FF0000160000000B
:1010E0000C000000F6FF00001200000025000000C8
:1010F00006000000060000002D0000002000000097
:10110000000000001C00000031000000070000008B
:10111000000000002900000017000000EBFF0000A5
:10112000060000001D000000EAFF0000DBFF0000D9
:101130000A000000F8FF0000C3FF0000E1FF00000C
:1011400002000000CBFF0000BBFF0000F7FF000023
:10115000ECFF0000B3FF0000DBFF00000C0000000C
:10116000D7FF0000C7FF00001400000014000000BB
:10117000D5FF000004000000450000000C00000046
:10118000F5FF00004E0000005000000001000000CC
:101190002D000000760000002E000000030000007B
:1011A0005F0000005D000000F4FF0000150000007B
:1011B0006200000008000000C5FF000025000000DC
:1011C00023000000A2FF0000BDFF00001B00000084
:1011D000B9FF000068FF0000DBFF0000EBFF00002C
:1011E0005EFF000082FF000003000000A8FF000077
:1011F00053FF0000E7FF00001600000083FF00001F
:10120000B4FF00005E0000000B000000A9FF00001A
:1012100059000000A1000000F7FF000022000000BC
:10122000E900000089000000FFFF0000B600000098
:10123000040100002600000030000000060100004C
:1012400086000000BAFF00006E000000C100000030
:10125000A4FF000086FF000079000000E4FF00000A
:10126000D9FE0000A2FF00001C000000D0FE00001C
:10127000A5FE0000E6FF000061FF00002DFE00005B
:1012800037FF00000F000000AAFE000087FE0000EC
:101290004D000000F3FF00008EFE0000F5FF00008F
:1012A0004D010000B3FF00007FFF0000E4010000DB
:1012B000A1010000B5FF0000670100004803000025
:1012C0000B0100005E0000007A0300000D03000027
:1012D000D5FF0000B9010000560400009500000091
:1012E000ABFE0000270300004E020000E2FB0000FE
:1012F00038FE000020030000F9FA00009CF4000012
:10130000C3FE000099FC000000DE000005D40000D0
:1013100000000000FA2B0000FE2100006603000020
:101320003D010000630B000006050000E0FC00002A
:10133000C70100001D040000B3FD0000DAFC00003E
:10134000550100006BFF0000ACFB000048FE0000F0
:101350002B000000F5FC000088FC0000A3FF00004B
:10136000F6FE0000BAFC00009AFE00004B000000F0
:1013700060FE00001EFE0000810000004C00000026
:10138000B4FE00000B000000710100000D00000021
:10139000B4FF00007701000055010000F1FF0000DC
:1013A000C8000000D10100009F0000001A000000EA
:1013B000590100002E010000E4FF00005E00000063
:1013C000250100001C00000087FF000079000000DC
:1013D0005C00000040FF000093FF0000450000009B
:1013E0007BFF0000FCFE0000D1FF0000DAFF0000E0
:1013F000FEFE00004CFF00000100000078FF00002E
:1014000019FF0000DFFF00000900000060FF00007E
:10141000A7FF000056000000F5FF0000A3FF00003A
:101420004C0000007C000000EAFF000019000000F2
:10143000AB00000057000000FDFF00007D00000031
:10144000A10000001500000025000000970000002A
:1014500047000000E5FF0000420000005D000000C2
:10146000DDFF0000DBFF00003A000000F9FF000094
:101470009FFF0000EBFF00000C000000A4FF000035
:10148000A2FF0000FDFF0000D3FF00008BFF000063
:10149000D3FF0000FFFF0000B1FF0000B3FF00001A
:1014A0000B000000F5FF0000BCFF0000FCFF000087
:1014B0002B000000EDFF0000ECFF000039000000F1
:1014C00029000000F4FF0000240000004C00000090
:1014D0001300000009000000440000003400000078
:1014E000FEFF00001E0000003C000000080000009D
:1014F000F6FF00002400000016000000E4FF0000DA
:10150000FAFF000015000000E9FF0000D8FF00000E
:1015100000000000F9FF0000D0FF0000E4FF000021
:1015200000000000E1FF0000D4FF0000FAFF00000F
:10153000FAFF0000DBFF0000EEFF00000A000000E1
:10154000F4FF0000EAFF00000B0000000F000000A5
:10155000F5FF0000030000001B0000000900000070
:10156000FEFF0000170000001A000000020000004B
:101570000A0000001C0000000C000000FFFF00003B
:101580001000000012000000FCFF0000FFFF000040
:101590000E00000000000000F4FF00000100000049
:1015A00004000000F2FF0000F5FF00000100000051
:1015B000F8FF0000EFFF0000FBFF0000FFFF00004E
:1015C000F2FF0000F5FF000001000000FBFF00003B
:1015D000F4FF0000FFFF000003000000FAFF00001E
:1015E000FCFF00000600000003000000FDFF0000FB
:1015F00005000000080000000100000001000000DC
:1016000009000000060000000000000005000000C6
:1016100007000000010000000000000005000000BD
:1016200003000000FEFF00000100000003000000B6
:10163000FEFF0000FDFF000001000000FFFF0000B2
:10164000FCFF0000FEFF000000000000FDFF0000A6
:10165000FCFF000000000000FFFF0000FDFF000095
:10166000FFFF000000000000FEFF0000FEFF000082
:101670000100000000000000FFFF0000000000006B
:101680000100000000000000000000000100000058
:101690000100000000000000010000000100000047
:1016A0000000000000000000010000000100000038
:1016B0000000000000000000010000000000000029
:1016C000000000000000000000000000000000001A
:1016D000000000000000000000000000000000000A
:1016E00000000000000000000000000000000000FA
:1016F00000000000000000000000000000000000EA
:1017000000000000000000000000000000000000D9
:101710000600FA001007980021079800213A80007F
:1017200000FE2F0000806000203A8800213A8000EF
:10173000F0F32F0000806000203A8800A002200013
:10174000303A8800007E2000001988002223EF0034
:101750002080200020198800404020004019880087
:10176000F0FC2F006019880021E3A8000468EF0056
:1017700085A0A9005105800000072000010070002D
:101780005005880095A0A8002023A8000070200024
:10179000503A8800F2E3A800F3E3A800F243A9005E
:1017A000F343A900811F800000F82F0080806000B3
:1017B000B003200001007000801F8800F103A80022
:1017C000F423EF00F823EF00F623EF00F1E3A80085
:1017D0008DE0A9008DC0A9009DE0A8009DC0A900D2
:1017E0000000EB00000F7800150037001E007800A5
:1017F0008000400080382800008040009000780081
:101800001E0078000001400080002100000041001F
:10181000010878001E0078008000400080782800D1
:1018200000804000900078001E0078000001400019
:101830008040210000004100010878001E0FE800F0
:10184000F01F20009E007800808F5000E7FF3400DA
:10185000FFFF370008080000001000000000000033
:101860000008000008000000000000000000000068
:10187000FFFFFF00FFFFFF00FFFFFF00FFFFFF0074
:10188000FFFFFF00FFFFFF00FFFFFF00FFFFFF0064
:10189000FFFFFF00FFFFFF00FFFFFF00FFFFFF0054
:1018A000FFFFFF00FFFFFF00FFFFFF00FFFFFF0044
:020000040001F9
:0200000401F009
:10000000FFFF0000FFFF0000FFFF00008100000075
:10001000A30000005F000000F7000000DFFF000009
:10002000FF000000FF000000FF000000FF000000D4
:00000001FF
